:030000000219FDE5
:03000B000200A848
:03002B0002015A75
:03005B000202EEB0
:030073000202DBAB
:1000800002030406080C10182030406080040608A3
:100090000C10182030406080A0C00003070F1F051F
:1000A000050D050305030302C2AFC0D0C0E0206206
:1000B00014E5256009E473E525F4F58AD262D0E001
:1000C000D0D0D2AF3285268AC262E526F4602F30C6
:1000D000682520720DD0E0D0D0C2B1C287C281D2D3
:1000E000AF32C2B1C287C281206F0C206609740A88
:1000F000D5E0FDE57B4280D0E0D0D0D2AF32758A2A
:1001000000C28DD26201F701B7306805206602D2C5
:10011000B101B7306805206602D28701B7306805A3
:10012000206602D28101B7C28230680A2066077455
:1001300008D5E0FDD2B101B7C28630680A20660753
:100140007408D5E0FDD28701B7C28030680A206606
:10015000077408D5E0FDD28101B7C2AFC2AD53E646
:10016000EFC0D0C0E0D2D3D2AFC2CEE52A60072024
:100170007449152A21BB7800790020742EE580305F
:100180007E01F430E50278FF53DACF207E0343DAB4
:1001900020307E0343DA10C2D8C271E580307E0180
:1001A000F430E50279FFC3E89970CB306103752A1A
:1001B00018207403752A18885CD27020740DE52B02
:1001C0006004152B21CB43DA01C2D8207002413ED6
:1001D000A85C206102C270207431C3E894F040032F
:1001E00074F0F8E8C4540F28F87984B70302410B7F
:1001F000C313C3138721200802C313200A06C3C8F0
:1002000098F8410B28F8500374FFF8C3E89565503F
:1002100003E565F88822E52D54066022206B1FE572
:1002200036C333C333F8E564C313C313F9C395224C
:1002300040028922E82522F52250037522FF8522FB
:1002400024A824C3E52495614002A8618825E566B9
:1002500070024182C3E8AA669A5003E8FAE4F9EA18
:10026000C333FBE568F45B29400D2567F8E567605B
:10027000021567400B41820AC3E5679A5002056781
:1002800078FF8826C26FC3E52694F84002D26FC378
:10029000E52594404002D26420CF0AD0E0D0D0437C
:1002A000E610D2AD32C2CF053A7801E52A600530BA
:1002B0007402152AC3E55C94014005755F0041D1C5
:1002C000756000756900E55F2401F55F5003755F97
:1002D000FFD0E0D0D043E610D2AD32C2AF53E67FBC
:1002E0007592FA7593FFC260759104D2AF32C2AFB6
:1002F00053E6EFC2ADC0D0C0E0C0F0D2D3D2AFA8B9
:10030000FBA9FCC2D8307102615553DACF207E03BD
:1003100043DA10307E0343DA20D271E580307E016B
:10032000F420E502612C88278928A18253DACF20A6
:100330007E0343DA20307E0343DA10C2D8C2713024
:100340007402A16E7800E580307E01F430E502A1F0
:100350006E885CA15653DACF207E0343DA20307ECC
:100360000343DA10C271206102812E53DACF207E5E
:100370000343DA10307E0343DA20C2D8D2718857A3
:100380008958C3E89555F8E99556F97B007E087AB7
:1003900000C3E8948CE994005005755B00812088C7
:1003A0002178A2E6A8216055C3E894C8E9940050DA
:1003B00008E4D2E4FB7A0A61FBC3E89468E994019B
:1003C0005008E4D2E3FB7A0F61FBC3E894D0E994D0
:1003D000025008E4D2E2FB7A1E61FBC3E894A0E974
:1003E00094055008E4D2E1FB7A3C61FBC3E89498A1
:1003F000E994085008E4D2E0FB7A787E00C3E895DF
:1004000059FCE9955AFD30E70AECF42401FCEDF4BF
:100410003400FD755B00C3EC9AED9E5003755B01E3
:100420008859895A8557558558567802A156C3E888
:100430009527F8E99528F9307C02A13A307B02A192
:100440003A307A02A1332075028151E9FDE8FC813E
:1004500070E9C313F9E813F8307902A133E9C31343
:10046000F9E813F8307802A133E9C313FDE813FC6F
:0F04700020612CC3EC941CED940240028187EDB7
:10047F00701EC3EC94C850180529E5297002152980
:10048F00C3E529940A5002A16E755C00D270A16E6B
:10049F00E529600215297888E6F97400207F08782D
:1004AF0096B90302789EE624FAFEE43400FFC3EC0B
:1004BF009EFCED9FFD9208B90310A208500720760D
:1004CF0009D27681D9307602C276A2085016B903C6
:1004DF000DECF42401FCEDF43400FD0204F378007C
:1004EF007900A13AB90315EC33FCED33FDC3EC945D
:1004FF000AFCED9400FD50047C007D00C3EC94FFDA
:10050F00ED9400400678FF7900A13AEC8572F0A4D3
:10051F00C5F0A2F733F87900400302055678FF794A
:10052F0000020556E9C313F9E813F8307C0EE960B1
:10053F000278FFC3E81338F8E43400F9C3E894FFF6
:10054F00E99400400278FF885CD270206102A16EAE
:10055F00741FF4552F4BF52FC274EB7002D27475C4
:10056F002A18307403752A0A306102A1822074039D
:10057F0053DAFE207403752B06D0F0D0E0D0D0D222
:10058F00AD43E6103279010205B279030205B27963
:10059F000A0205B2791E0205B279640205B279C862
:1005AF000205B27817E4D5E0FDD8FAD9F6227A140D
:1005BF007B780205D97A107B8C0205D97A0D7BB432
:1005CF000205D97A0B7BC80205D97902E4C286D518
:1005DF00E0FDD287D5E0FDC287D5E0FDD286D5E01C
:1005EF00FDE920E002D2B130E002D281E573D5E01F
:1005FF00FDE920E002C2B130E002C2817496D5E07D
:10060F00FDD9C9EAF8D5E0FDD8FBDBBEC28622C30F
:10061F007C007D0075F00005F0EA33FAEB33FB50F8
:10062F00F6EB13FBEA13FAC3E9FFE8FEE89AF8E9E1
:10063F009BF95004EFF9EEF8B3EC33FCED33FDD535
:10064F00F0DFEDF9ECF822E889F08A20D2D4F8A98E
:10065F00F07B0030F70B7BFFF42401F8E9F4340052
:10066F00F9E88520F0A4ADF0F8E98520F0A4AFF00B
:10067F00FEED2EF974003FFA7C04C3EA13FAE91376
:10068F00F9E813F8DCF48BF030F70AE8F42401F8FA
:10069F00E9F43400F9E889F0C2D4F8A9F02222C3B2
:1006AF00E54113F9E54013F8C3E54498F8E545999A
:1006BF00F9500CC3E89480E994FF40160206E5C395
:1006CF00E8947FE9940050030206E5787F790002F1
:1006DF0006E5788079FF8849894A22E5492546F859
:1006EF00E54A3547F9854A20E4300701F43548FAE1
:1006FF0030E709C3EA94F04015020723C3EA940FC9
:10070F00500302072378FF79FF7A0F02072378003F
:10071F0079007AF0C3E5249561500AC374019524DA
:10072F00500B020741E54A20E70E020741E54A3028
:10073F00E706884689478A482278A5E6FAC3E5493D
:10074F0033F8E54A33F9D156E930E70BC3E8948023
:10075F00E994FF4013E17BC3E8947FE994005002D2
:10076F00E17B787F7900E17B788079FFE820E715DE
:10077F00C3E52398F84009C3E8940140030207A298
:10078F0078010207A2E8F424012523F840030207A9
:10079F00A278FF884B2278A6E6FAA847A948D15637
:1007AF00E930E70CC3E89401E994FF40160207D63D
:1007BF00C3E894FFE9940050030207D678FF79004D
:1007CF000207D6780179FFE920E715C3E54B98F8C2
:1007DF004009C3E8940140030207FD78010207FDB9
:1007EF00E8F42401254BF840030207FD78FF882425
:1007FF002278FFC26420693D206A12D264C3E541AA
:10080F00940A4009C3E52594405002C26479A1E7D8
:10081F006023E541601F74FF8541F0848539F03016
:10082F006A0375F005A4F8C5F0600278FFC3E89578
:10083F00645002A864886322C3E5409440E5419464
:10084F0001E5635003140158046002F563220208A6
:10085F00602275E890227883E6FFE5E820ECF7A8A0
:0F086F00BDA9BE0570C3E57094084052757000B6
:10087E00E9FA79A0E76044EA7007E571601B0208A7
:10088E009BC3E895716010E5715006600C14020868
:10089E00A70460F90208A7E571F571C394A8401B7F
:1008AE007561C0C394054013756180C39405400BF8
:1008BE00756140C39405400375610075BB0622E562
:1008CE0061F460020561E570B4070375BB1E227406
:1008DE003279A787F0A4C5F0A2F733F8C3E8956183
:1008EE004002A8618822882488258826886422757B
:1008FE0040007541F022C2AF75C820A8CCA9CDAA80
:10090E003A30CF010A75C824D2AFAB3BAC3C883B22
:10091E00893CC3E89BF8E99C206908F930670241DD
:10092E0010216DAD3D8A3DF9EA9DFA600478FF799C
:10093E00FFAE3EAF3F8B3E8C3FA83BA93CC3E89E2B
:10094E00F8E99FF9C3E54113FBE54013FAE82AF5F0
:10095E0040E93BF54150067540FF7541FF21B7AAAE
:10096E0040AB41AC40AD417E047F02C3EB940440EA
:10097E00021E1FC3EB940840021E1FC3ED13FDECB5
:10098E0013FCDEF7C3EA9CFAEB9DFBEF6009C3E9AB
:10099E0013F9E813F8DFF7EA28FAEB39FB8A408BF4
:1009AE004150067BFF8B408B41C3EB94025002D229
:1009BE00673069047F0321E27892E6FFC3E537943E
:1009CE008240110FC3E53794A040010FC3EF940688
:1009DE0040027F057E02E541C4540FF9E541C4543F
:1009EE00F0F8E540C4540F28F8C3E89EFAE99400E5
:1009FE00FB4009C3EA9402EB940050047A02E4FB34
:100A0E00415CAA40AB41EBC4FEEAC4540F4EFCC39A
:100A1E00EA9CFAEB9400FBC3E813C313F8EA28FA36
:100A2E00EB3400FB8A408B41C3EB94024002C26759
:100A3E007802EBC4FE7B00EAC4540F4EFAC3EA9868
:100A4E00FA4005C3940250027A027892E6FF3060B3
:100A5E0002415C855192855293D26043E680C3E495
:100A6E009AF8E49BF930670241E8E8FAE9FBD3E92A
:100A7E0013FDE813FC88518952C3EF94036038EFDD
:100A8E0020E00DE82CF8E93DF9ECFAEDFB020AB195
:100A9E00E828F8E939F9C3E82402F8E93400F97ACC
:100AAE00FE7BFFC3EF9403400E8A538B54884D890F
:100ABE004E8C4F8D50611C885389548A4D8B4E8CB1
:100ACE004F8D503069127553F07554FF754FF07598
:100ADE0050FF7551F07552FF611CE8FAD3E813FC14
:100AEE008851C3EF94036020EF20E007E82CF8EC68
:100AFE00FA6108E8282402F87AFEC3EF940340084E
:100B0E008A53884D8C4F611C88538A4D8C4FE568F3
:100B1E00C3335002646BF56830600261267534028F
:100B2E00D26043E680E52D54066034A840A941C347
:100B3E00E913F9E813F8C3E913F9E813F830690477
:100B4E00E92440F9C2AF53E67F759100C3E498F5EE
:100B5E0094E499F595759104D26043E680D2AF2264
:100B6E00D265754300752000306C03752040020B72
:100B7E008DD265754300752040306C03752000786A
:100B8E00017901206720E52D54066002C2657914B3
:100B9E00E541C313700104F8C39414400278143075
:100BAE006904781B791B206010E543600C306903E3
:100BBE00D53404D26D812F712E0543E59B5440B57B
:100BCE002002811930690908C3E89940011861B4FF
:100BDE0020650A08C3E8994002618D61B4C265C2FE
:100BEE00AF53E67F7591003067127594007595FED0
:100BFE00759104D26043E680D2AF618DAE40AF41B5
:100C0E00C3E49EF594E49FF59561FEC3E53394012C
:100C1E005002618D306502618DD802812D61B4C2A2
:100C2E006DC2AF53E67F75910085539485549575CB
:100C3E009104854D92854E93D26043E680D2AFE506
:100C4E002D54066008206A020533020C6B306D0DC0
:100C5E00206C0A2065071581158102152222780065
:0F0C6E003064053065027801E53775F007A4F9A9
:100C7D00E5F028F5F0E9A2F013A2F113A2F213F5B5
:100C8D0037C394785003753778C3E53795384008E6
:100C9D00D266C2B1C287C28130600281A5854F92F2
:100CAD00855093D26043E68022207D16C2AF7542F7
:100CBD0002C286D282306202D281D2AF759F020209
:100CCD000EA5C2AF754202C286D280306202D2B189
:100CDD00D2AF759F02020EA5307243207D20C2AFA8
:100CED00754203900138757B40C281C28030620429
:100CFD00D287A103D286D2AF759F03020EA5C2AFD4
:100D0D00754203900138757B40C2B1C282306204D6
:100D1D00D287A123D286D2AF759F01020EA5207D69
:100D2D0017C2AF754203900113C281306202D287A0
:100D3D00D2AF759F03020EA5C2AF7542039001138A
:100D4D00C2B1306202D287D2AF759F01020EA520CB
:100D5D007D16C2AF754204C282D280306202D28744
:100D6D00D2AF759F01020EA5C2AF754204C280D2EB
:100D7D0082306202D287D2AF759F03020EA5307208
:100D8D0043207D20C2AF754205900127757B04C2BB
:100D9D0087C286306204D2B1A1A9D282D2AF759F2B
:100DAD0002020EA5C2AF754205900149757B01C2C5
:100DBD0087C286306204D281A1C9D280D2AF759F1D
:100DCD0002020EA5207D17C2AF754205900109C222
:100DDD0087306202D2B1D2AF759F02020EA5C2AFAB
:100DED0075420590011DC2873062EBD281D2AF757D
:100DFD009F02020EA5207D16C2AF754206C280D29B
:100E0D0086306202D2B1D2AF759F03020EA5C2AF7A
:100E1D00754206C282D286306202D281D2AF759FF0
:100E2D0001020EA5307243207D20C2AF75420190A4
:100E3D000149757B01C2B1C282306204D281C14FBA
:100E4D00D280D2AF759F01020EA5C2AF754201903F
:100E5D000127757B04C281C280306204D2B1C16F9B
:100E6D00D282D2AF759F03020EA5207D17C2AF753A
:100E7D00420190011DC2B1306202D281D2AF759F85
:100E8D0001020EA5C2AF754201900109C281306207
:100E9D0002D2B1D2AF759F03C26622900107757B56
:100EAD0000C2B1C287C281C282C286C280C2622222
:100EBD00788076FF0876FF0876FF0876FF087603C0
:100ECD000876040876090876030876010876017815
:100EDD008C76010876FF0876FF0876FF0876FF0806
:100EED0076FF0876030876FF0876FF0876FF08760A
:100EFD00250876D00876FA0876FA0876040876FF83
:100F0D0008760108760008767A0876FF08760108DB
:100F1D007601087600087603087600227887E6FFCA
:100F2D00C272BF0302D2727888E6C394036008C20E
:100F3D007DE630E102D27DC27E7889E630E102D2D3
:100F4D007EC3EF94026008758E01D273020F617536
:100F5D008E00C273227880E6149000809378A5F6F7
:100F6D007881E6149000809378A6F67886E6149042
:100F7D00008D9378A7F67886E6F539C39402500371
:100F8D00753902789CE67538FFB402037538A0B444
:100F9D00030375388278A3E61490009A93F566D111
:100FAD00A822C2B3789DE66002D2B3227896E6FA03
:100FBD007897E6FB7888E6B40305C3EB940EFB3017
:100FCD007F047A007BFFC3EB9AFCC3948250027CB2
:100FDD00827572000572EC8572F0A4C3E5F0947D04
:100FED0040F222D27FF1B91205A37A007B007C106A
:100FFD00120599E55C2AFA74003BFBDCF37C04C313
:10100D00EB13FBEA13FADCF7FEC27F120FB922E5F0
:10101D00EF20E6037520000520903DFFE5201460CC
:10102D0006901FFF1460009304600375EF1253D9EF
:10103D00BF7581C043FF8012059475EF0243B20363
:10104D00E5B3240220E70DF521E5B120E006852169
:10105D00B343B101120EA875803875A4C775F1FFA1
:0F106D0075D4DF7590FF75A50075F20075D5007D
:10107C0075A0FF75A60075F30075D60075B0E47504
:10108C00A71B75F4FF75E241120EA8E4F8F6D8FD23
:10109C00756801120EBD1215737898867375300140
:1010AC00C2AF1205AD1205BD1205A31205C412057F
:1010BC00A31205CB1205A312168C1205AD1205ADA9
:1010CC001205A8C2AF78FA79FA308507D9FBD8F7A0
:1010DC00021C00120F29120F62120FAF120FB978F7
:1010EC00988673120EA875881075890275C82475B8
:1010FC00910475D84075A82275B80275E690759B59
:10110C0080759D0075D10E75BC5875BB0675BA1FE0
:10111C0075E880120594D2AF12085D75360053DA6B
:10112C00CF207E0343DA20307E0343DA1043DA010A
:10113C00C2D8C2711205ADD2617B037A0CE55B702B
:10114C00077A0CDB030210CF1205A32070030210E8
:10115C00CFC270E55CC3940240E1E52F541F855E5D
:10116C005DF55EB55DD5DAD5C26153DACF207E036D
:10117C0043DA20307E0343DA10C2D8C27178A2E67B
:10118C007008D274E52F54E0F52FC2757529001242
:10119C0005A8307409C3E529940A4002D2751205DA
:1011AC009978023074027800C3E55C9840F0C2AFC5
:1011BC001205BD1205BD1205BDD2AF1205AD754CA1
:1011CC00007888E6B4030241B2120599788CE6C324
:1011DC00940150030212B2E530C394015003021281
:1011EC00B2207435C3E55C94FF50030212B2C2AF57
:1011FC001205D2D2AF1205A8C3E55C940150EFC220
:10120C00AF1205BD12059E1205BDD2AF1205A8C3C3
:10121C00E55C94FF40E90217117F05D27F120FB9EC
:10122C001205A8C2AFC27F120FB9AE5CC3E55C94C5
:10123C007FD2AF407B120594C2AF1205D2D2AFDF82
:10124C00DA120FF0C3EE94057897F61205AD12156D
:10125C00B51216947F0AD27F120FB91205A8C2AF2D
:10126C00C27F120FB9AE5CC3E55C947FD2AF50E481
:10127C00120594C2AF1205BD12059E1205BDD2AF68
:10128C00DFD4120FF0EE24037896F61205AD12158A
:10129C00B51216C31205A8120FB9C3E55C94FF5022
:1012AC000221ED021711C3E55C954C4003855C4CA3
:1012BC001205A878017988E7B403027805C3E55CC8
:1012CC0098400221CDC2AF1205D21205D21205D21E
:1012DC00D2AF1205AD753000E4F531F5320531E5CC
:1012EC0031F4703F0532789AE6781914601278322E
:1012FC0014600D787D14600878FA14600375320060
:10130C00C3E53298401D120EA812059415327531A2
:10131C000078998673C2AF1205D2D2AF78988673D3
:10132C001205A812059EE52A700530740201CF78CB
:10133C00012074027806C3E55C9840A17888E6C366
:10134C00940360031205A8E52A70030210CFC2AF04
:10135C00120EA8E4F522F523F524F525F526F567FC
:10136C00D2AF7885E6C333F565E4F544F545F5462B
:10137C00F547F548F570F52CF52DF53775700875B2
:10138C00BB1E120594120861E5E820ECFBA8BDA970
:10139C00BEE97001F8887112086575700875BB1E7E
:1013AC00120F29C2AF7561FF1208DD8522618522FB
:1013BC0062852263D2AF75220175240175250175F2
:1013CC002601856069756A017888E6B40307C27DD9
:1013DC00307602D27DD268D269753300120E0212B9
:1013EC000E311208FD1209041208FD12090412082C
:1013FC00FD120B7F1206AD120C6C120CB612090406
:10140C00120B6E306E031206AE206703120800300A
:10141C006703120847120C6C120CE5120904120B2C
:10142C007F306E031206EA120C6C120D5C1209046A
:10143C00120B6E306E03120748120C6C120D8B12CD
:10144C000904120B7F306E031207A5120C6C120EDE
:10145C0002120904120861120B6E120C6C120E317E
:0F146C0012086512090430692F85646185646276
:10147B00856069756A0179187A0CC3E53399400C5C
:10148B00C269D26A8A357561FF0214A4C3E55C9404
:10149B000140030213FD02152A306A1D206C1AE568
:1014AB0035147006C26AD26B61FDF535C3E55C94E9
:1014BB000140030213FD02152A753600788279A4C8
:1014CB00E760027803C3E55F985054307404E52A53
:1014DB00604D7888E6B40317207D0520760781FAE6
:1014EB0030760281FA206C07D26C856461813C787E
:1014FB00F0306C058564617820C3E541985002613A
:10150B00FD306C1BC26CC27D307602D27DD26A7507
:10151B00351285646161FD0536E55C6002A12D75B0
:10152B003600C2AF120EA87887E6FE7602120F299C
:10153B007887EEF6E4F522F523F524F525F526F567
:10154B0065752C00752D00D2AF1205A8120EA87868
:10155B00A4E66006D2B1D287D281307409C3E536D6
:10156B009404400201CF41E4901A0D78201215F734
:10157B00E520B45A0CA31215F7E520B4A503021508
:10158B0095120EBD1215B50215B4901A0378807B17
:10159B000A1215F7A308DBF9901A0F788C7B191236
:1015AB0015F7A308DBF9901A2822C2AF12163612D0
:1015BB001610901A00740E1215FCA374061215FC6B
:1015CB00A374151215FC901A0378807B0A1215FB75
:1015DB00A308DBF9901A0F788C7B191215FBA30863
:1015EB00DBF9121649121627901A2822E493F622D9
:1015FB00E6438F01538FFD75EF0275B7A575B7F1F4
:10160B00F0538FFE22438F02438F0175EF0275B7A4
:10161B00A575B7F1901A0DF0538FFC22901A0D742B
:10162B005AB1FC901A0E74A5B1FC227A3079D0789D
:10163B0020901A40B1F7E520F709A3DAF7227A30A8
:10164B0079D0901A40E7B1FC09A3DAF922AB74A860
:10165B0075BB01027984BB02027985BB03027986D3
:10166B00BB04027992BB05027987BB060279A3BB47
:10167B000702799CBB08027988BB09027989E8F7D4
:10168B00227C051205ADDCFB22C2AF1205BD120593
:10169B00C41205CB1205D212059E1205BD1205C44C
:1016AB001205CB1205D212059E1205BD1205C412EE
:1016BB0005CB1205D2D2AF22C2AF1205D21205CB87
:1016CB001205C41205BD12059E1205D21205CB12CE
:1016DB0005C41205BD12059E1205D21205CB1205CB
:1016EB00C41205BDD2AF22AE74AF75C2AF1205BD29
:1016FB001205BD1205BD12059EDEF21205D21205B2
:10170B009EDFF8D2AF22D194D18CD18C7574017538
:10171B007501757600D1F27C05AD5C1205ADC3ED9C
:10172B00955C70F5C3E55C9401400AC3E55C94FFDE
:10173B00403202174DD158B1B5D194C2AF75EF12EB
:10174B00D18CDCD50576C3E5769403500280C6D1E7
:10175B008C0575E5741490009F93F808C3E5759894
:10176B00500280AED18CD18C0574C3E574940A50B1
:0F177B0002809C120EBDB1B5C2AF75EF12D18CBA
:0319FD0002101CB9
:101A00000E0615FFFFFFFF0304090301015AA5019C
:101A1000FFFFFFFFFF03FFFFFF25D0FAFA04FF01DE
:091A2000007AFF0101000300FF40
:101A4000235475726E6967794145343541232020EE
:101A500023424C48454C4923463331302320202033
:101A60002020202020202020202020202020202076
:101C0000C2AFC2D353D9BF7581C043B20343FF8073
:101C1000752438752503B1C975EF0275E24043F1AB
:101C20002053A4DF75D4FFD2857DFA780379E67C52
:101C300010752200752300901DD67B0675249875BB
:101C400025013085028142208508D8FBD9F9DCF7CF
:101C500081B4308508D8FBD9F9DCF781B4B189E4C7
:101C600093A3C39A6004DDC381B4DBDBB17B600264
:101C7000812B7B08E493FAA3B15CDBF87A30B15C8A
:101C8000752200752300B17BEAFCEBFDC3ED94FEE9
:101C9000400EB17B8A278B28ED30E0048A828B834B
:101CA000B17B7AC270D8C3ED94FE601350CEBD00F4
:101CB00025EC60097520007521FF0200008100A855
:101CC00027A9280809D804D90281D3B17FEA89AAB3
:101CD000F281C50D81A0C3ED94035049EDA2E092BD
:101CE000007AC5C3E5829400E583941C50902000DF
:101CF00010438F02438F0175B7A575B7F1F030001F
:101D00001FA827A9280809438F01538FFDD804D99C
:101D100002A12089AAE275B7A575B7F1F0A3A10DBC
:101D2000538FFC817C7AC1BD030CE493A3FAB140CC
:101D3000DCF8B138817C817EAA22AB23B15CEBFA5E
:101D4000EA6222752608C3E52313F523E52213F57D
:101D50002250066323A0632201D526EAB1C9B1C986
:101D600075260AEAF4200102D285300102C285B14B
:101D7000C9C3134002C201D526EB22B17FEAFB2082
:101D80008502A17F308502A184752608AE24AF2587
:101D9000C3EF13FFEE13FEB1CDB1C9C3EA13308513
:101DA000024480FA30E703632201C3E52313F523DD
:101DB000E52213F52250066323A0632201D526D91C
:101DC000E52265236523F52222AE24AF250E0FDE22
:101DD000FEDFFCD20122424C48656C693437316326
:041DE000F3100601F5
:00000001FF
